:100000000C94B2020C94EA020C94EA020C94EA02F8
:100010000C94EA020C94EA020C94EA020C94EA02B0
:100020000C94EA020C94EA020C94A8270C947C2805
:100030000C9479220C94EA020C94EA020C94EA02E1
:100040000C94EA020C94EA020C94EA020C94EA0280
:100050000C94EA020C9400230C94EA020C94EA0239
:100060000C94EA020C94EA020C94EA020C94EA0260
:100070000C94EA020C94EA020C94EA020C94EA0250
:100080000C94EA020C94EA020C94EA020C94EA0240
:100090000C94EA020C94EA020C94EA020C94EA0230
:1000A0000C94EA020C94EA020C94EA0229001E0065
:1000B0001F0020002100220023002400250026002C
:1000C00027002D002E002A0000002B0014001A002B
:1000D0000800150017001C0018000C001200130087
:1000E0002F00300031004B003900040016000700DB
:1000F00009000A000B000D000E000F003300340051
:10010000000028004E00E1001D001B000600190041
:100110000500110010003600370038000000000014
:1001200052000000E0000000E20000002C00E300AC
:1001300001510000000090000000500051004F00ED
:100140004C0001003A003B003C003D003E003F00F7
:10015000400041004200430044004500010000000F
:10016000010000000000000000000000000000008E
:100170000000000000000000000000004A00010034
:10018000000000000000000000000000000000006F
:10019000000000000000000001004D000100000010
:1001A000000000000000000000000000000000004F
:1001B000000000000000010000000100000001003C
:1001C000000001000100010000000000000000002C
:1001D00001000100010046001E0F0500047F3F1FC3
:1001E000643214643214783C1E1E140A052223253E
:1001F0002628292A2C2D2F3032333536383A3B3DEC
:100200003E4042434547494A4C4E50515355575939
:100210005A5C5E6062646668696B6D6F7173757756
:10022000797B7D7F81838587898A8C8E9092949655
:10023000989A9C9E9FA1A3A5A7A8AAACAEAFB1B364
:10024000B4B6B8B9BBBCBEBFC1C2C3C5C6C7C9CAB4
:10025000CBCCCDCED0D1D2D2D3D4D5D6D7D7D8D976
:10026000D9DADADBDBDBDCDCDCDCDCDDDDDDDDDCD4
:10027000DCDCDCDCDBDBDBDADAD9D9D8D7D7D6D5E6
:10028000D4D3D2D2D1D0CECDCCCBCAC9C7C6C5C3A8
:10029000C2C1BFBEBCBBB9B8B6B4B3B1AFAEACAAF5
:1002A000A8A7A5A3A19F9E9C9A98969492908E8CA5
:1002B0008A89878583817F7D7B79777573716F6D7F
:1002C0006B6968666462605E5C5A59575553515059
:1002D0004E4C4A4947454342403E3D3B3A3836350D
:1002E0003332302F2D2C2A292826252322FFAA7FBE
:1002F0005540000101010101010101010202020258
:1003000002020202020303030303030303040404BF
:100310000404040405050505050606060606070788
:1003200007070708080808090909090A0A0A0B0B40
:100330000B0C0C0C0D0D0D0E0E0E0F0F0F101011DF
:100340001111121213131414151516161717181865
:1003500019191A1A1B1B1C1D1D1E1E1F20202122CD
:1003600022232424252626272829292A2B2C2D2D13
:100370002E2F30313232333435363738393A3B3C30
:100380003D3E3F404142434445464748494A4C4D23
:100390004E4F50515354555658595A5B5D5E5F61EC
:1003A0006264656668696B6C6D6F7072737577787F
:1003B0007A7B7D7E8082838587888A8C8E8F9193DD
:1003C0009596989A9C9EA0A2A3A5A7A9ABADAFB104
:1003D000B3B5B7BABCBEC0C2C4C6C9CBCDCFD1D4E9
:1003E000D6D8DBDDDFE2E4E7E9EBEEF0F3F5F8FA8F
:1003F000FDFF1C03570049004E004700530020003A
:1004000048004F00540053005700410050000000C6
:100410000A0359004D0044004B0000000403090486
:1004200009023B00020100A0FA09040000010301D7
:100430000100092111010001224000070581030884
:10044000000109040100010300000009211101005D
:100450000122B600070582032000011201000200FC
:100460000000084D5975490100010200010501090C
:1004700002A10185020901A1000509190129081538
:100480000025019508750181020501093009311522
:1004900081257F95027508810609381581257F958C
:1004A0000175088106050C0A38021581257F950122
:1004B00075088106C0C005010980A10185031901E5
:1004C0002AB700150126B700950175108100C005F7
:1004D0000C0901A101850419012AA002150126A019
:1004E00002950175108100C005010906A10185066C
:1004F000050719E029E71500250195087501810216
:100500000507190029EF1500250195F075018102F5
:1005100005081901290595057501910295017503D5
:100520009101C005010906A101050719E029E71598
:100530000025019508750181029501750881010565
:1005400007190029FF150026FF0095067508810090
:100550000508190129059505750191029501750395
:100560009101C00011241FBECFEFDAE0DEBFCDBF86
:1005700004B603FE18C08091990590919A05A09148
:100580009B05B0919C058730904BA740B04B59F428
:100590001092990510929A0510929B0510929C0555
:1005A000E0E0F8E3099511E0A0E0B1E0E4EFF7E561
:1005B00002C005900D92A03DB107D9F725E0A0ED4E
:1005C000B1E001C01D92A939B207E1F70E9476128D
:1005D0000C94E22B0C94000081E0089581E00895D2
:1005E0000E94EE02089508950E94F3020895A5E086
:1005F000B0E0EDEFF2E00C94DD2A49835A833091AC
:10060000D30189819A81311119C0662399F022237F
:1006100089F00E942809182F682F89819A810E94E9
:10062000040969817A81812F0E94B80F2596E3E041
:100630000C94F92A0E941609182FF3CF0E9428095A
:1006400069817A81F1CFFC01262F4081518162813D
:10065000738184810E94F702089581E00895CF9309
:10066000DF93EC0160E00E942303BE010E94F402CC
:10067000DF91CF9108950E94F71008950E94FB101A
:10068000089508950E9453070E9441032FEF84E3C9
:100690009CE0215080409040E1F700C000000895A8
:1006A0000E9442030E94242308950E9442030E9454
:1006B000482308950F931F93CF93DF938C0161E03C
:1006C0000E942303EC01B8010E94F002811106C0D0
:1006D00080E0DF91CF911F910F910895B801CE0175
:1006E0000E94C61D8823A1F3B801CE010E94AA2052
:1006F000882371F3B801CE010E94DF1E882341F3E5
:10070000B801CE010E941C20882311F3B801CE014C
:100710000E94141C8823E1F2F8018281882361F091
:10072000CB35FDE5DF0701F158F4C115ECE5DE0737
:1007300091F0CF3DDC4591F0C8010E94EC02C9CF99
:10074000CD358DE5D80769F090F0C83ADD45A1F7C1
:100750000E945503BDCF0E945003BACF0E94EE0DF8
:10076000F7CF0E94280DE8CF0E94320DE5CF0E94FE
:10077000360DE2CF0E94552280E00E94FB1D0E94B0
:10078000EC030E947A1A08950E94F21C0E94F00362
:100790000E94511B0E945A22089508950E94CD0381
:1007A000089581E00895CF93C82F0E94D103882334
:1007B00019F0C1FD03C0479ACF9108954798FCCF27
:1007C0003F9A479A0895CF93C82F0E94CE038C2F4B
:1007D0000E94D303CF91089580E00E94E30308951F
:1007E0000E9406210E94E30308950E940621909131
:1007F000D201981721F08093D2010E94E30308955B
:10080000ABE0B0E0E6E0F4E00C94DE2A4F835887DA
:1008100069877A878B8761110E94730C1E821D8203
:1008200085E0FE013796DE01119601900D928A95C2
:10083000E1F78C819D81892B61F449815A816B811B
:100840007C818D819E810E949C0B2B96E2E00C9412
:10085000FA2A89819A8189238F3F79F3CE01019603
:100860000E942D038111E9CFF0CFFC01808191819D
:100870000E9462090895CF93C82F8823B9F08CEFA6
:100880008C0F813AA8F46C2F80910401909105019E
:100890000E947B21882329F08C2F0E94330C0E9418
:1008A000940C8C2F0E942B0C0E94940CCF910895D5
:1008B00080E28C0F883048F4C77081E001C0880F57
:1008C000CA95EAF70E94560CEFCFEBE5EC0FE33048
:1008D00040F4F0E0E45AFE4F808190E00E943B211A
:1008E000E5CFE8E5EC0FE73150F4F0E0EE0FFF1F45
:1008F000E25DFE4F808191810E945121D7CFCD3E94
:10090000A8F28C2F0E94FA120E94CD13CFCF882319
:1009100079F19CEF980F913A28F40E94330C0E94D1
:10092000940C089590E2980F983050F4877091E0FD
:1009300001C0990F8A95EAF7892F0E945C0CEFCFCE
:100940009BE5980F933028F490E080E00E943B21D3
:10095000089598E5980F973128F490E080E00E9480
:10096000512108958D3E20F00E9454130E94CD1312
:1009700008951F93CF93DF93182FEB010E943B0440
:10098000209739F4812F0E948704DF91CF911F9126
:1009900008958FE99FE00197F1F700C000002197CB
:1009A000EFCF70E060E0893311F460E570E00E9401
:1009B000B9040895882321F00E94560C0E94940CDB
:1009C0000895882321F00E945C0C0E94940C0895E5
:1009D000B0E0A0E0EEEEF4E00C94D72A6C01D62F44
:1009E000C72FFC011281F580F2949FE0F9220E944A
:1009F0004C0CE82E8823B9F0E12E1123A1F08C2FA6
:100A0000807F803421F080E28D0F8830D0F080919B
:100A10007D0482FF16C082E00E94F70C0E944C0CFD
:100A200091E0E82EE926BC2EB2948FE0B822FBE0DC
:100A3000FB1508F468C0EB2DF0E0EC51F44D0C947C
:100A4000972AE12CF0CF0C2F0F70C07F11F0029588
:100A5000007F112399F0002359F080E28D0F883038
:100A600010F0D11107C0802F0E94560C0E94940CE8
:100A70008D2F41C0802F0E94660CF8CF8D2F0E94D1
:100A80008704002309F43FC080E28D0F883010F006
:100A9000D11104C0802F0E945C0C03C0802F0E94E3
:100AA0006C0C0E94940C2FC00C2F0F70C07FC032B2
:100AB00011F00295007FDD2381F0D13009F463C08D
:100AC000112309F46DC0FF2009F463C0F60185818C
:100AD00080FFCECF8F7085835CC080917D0482FDC6
:100AE00033C0112359F0002329F0802F0E94560CA7
:100AF0000E94940C80E00E943B0405C080E00E94AC
:100B000087040111C7CFEB2DE850FF0B349720F479
:100B10000E9406210E94E303EE2089F00E94480C07
:100B200080FD0DC0F60112820E94420C0E940C084A
:100B3000C6010E9413070E94420C0E942E08CDB7E6
:100B4000DEB7E9E00C94F32A112389F0F11006C016
:100B50000E94760C802B0E94DA04D5CF21E0F2129D
:100B6000F7CF0E94760C802B0E947D0CCCCFF11029
:100B700006C00E948A0C802F0E94E104C4CF31E09D
:100B8000F31609F2F6CF112331F085E08F1508F442
:100B9000BACF802FE0CF94E09F1508F4B4CFEBCF0D
:100BA000FF2049F3D93349F4FFEF27EE33E0F1504A
:100BB00020403040E1F700C000008D2F0E948704E4
:100BC000A2CF8C2F86958695837069F0813009F0CD
:100BD0009ACF8D2F9C2F9370111102C090E080E06E
:100BE0000E94512190CF8D2F9C2F9370111102C024
:100BF00090E080E00E943B2186CF8D2F112329F0C9
:100C00000E94FA120E94CD137ECF0E945413FACF95
:100C10008C2F837009F041C0111175CF4D2F429573
:100C200046954770440F440F0D2F0F7010E030E0D1
:100C300020E0042E04C0000F111F221F331F0A944E
:100C4000D2F760E070E0CB01D4FF0FC06FE070E03E
:100C500080E090E004C0660F771F881F991F4A95B7
:100C6000D2F76095709580959095C695C695C3709E
:100C7000602B712B822B932BC23049F058F4C1307A
:100C800019F00E94B7073FCF0E94A4073CCF0E94F3
:100C9000CA0739CF0E94A10736CF8695112311F0DC
:100CA0008C2F8170882309F42ECF4D2F42954695C5
:100CB0004770440F440F0D2F0F7010E030E020E01C
:100CC000042E04C0000F111F221F331F0A94D2F7F5
:100CD00060E070E0CB01D4FF0FC06FE070E080E017
:100CE00090E004C0660F771F881F991F4A95D2F7BE
:100CF0006095709580959095C695C695C370602B4C
:100D0000712B822B932BC23049F058F4C13019F06B
:100D10000E948708F8CE0E947408F5CE0E949A08B7
:100D2000F2CE0E94E307EFCECF70112329F08C2F73
:100D30000E940C088D2F0FCF8D2F0E94E1048C2F65
:100D40000E942E08E0CED23F51F160F4D03FB9F0BE
:100D5000D13F81F0112309F449C0F11089CE8C2FC5
:100D60008F7121C0D33F11F1D43FA1F780917D0451
:100D700082FD26C08C2F8F71112311F314C0112313
:100D800049F084E08F1508F4BECE8C2F8F710E943D
:100D90005208B9CE95E09F1508F4B5CEF6CF8C2F4A
:100DA0008F711111CDCF0E940C08ADCE112329F007
:100DB0008C2F8F710E94F607A6CE0E94F007A3CE5B
:100DC000112349F0CF718C2F0E940C0863E08C2F07
:100DD0000E94D90C98CE81E00E94F70CE1E0EF155B
:100DE00008F091CE82E00E94F70C8DCEF110DACEA1
:100DF0008C2F8F71A5CF0F931F93CF93DF93EC01AF
:100E0000688179818A810E946D098C010E94AD08F8
:100E10000E94A007B801CE010E94E804DF91CF91A3
:100E20001F910F910895CF93DF93EC018B819C81EB
:100E3000892B29F08881998189238F3F51F4DF9193
:100E4000CF910895CE010E94FB06CE010E942F0390
:100E5000F6CFCE010E945A038111F4CF0E944C0CB0
:100E6000882369F38A81882351F380917D0482FF6E
:100E7000E6CF82E00E94F70CE2CF90E080E00E9493
:100E80003B2190E080E00E9451210E94730C0E945F
:100E9000940C0E94DE140E94CD1308950E943B0C16
:100EA0000E943D0708950E94630C0E944E0708951A
:100EB00092959F70963091F058F4925F9F709230A7
:100EC00058F4803F19F030F4883E30F481E0089502
:100ED0009A5FF4CF843FD1F380E00895883EB0F369
:100EE000813FD1F7F3CFFC01808191810E9462099B
:100EF0000E9458070895A5E0B0E0E1E8F7E00C94FF
:100F0000DE2A2596E2E00C94FA2AA6E0B0E0EBE8AF
:100F1000F7E00C94DE2A2696E2E00C94FA2A089573
:100F20000E948F0708950E94900760930A027093B1
:100F30000B0280930C0290930D020E943D070895CE
:100F400008950E94930708950F931F9300910A023A
:100F500010910B0220910C0230910D02602B712B2D
:100F6000822B932B0E9493071F910F9108950F934B
:100F70001F9300910A0210910B0220910C023091F4
:100F80000D0260237123822393230E9493071F91F4
:100F90000F9108950F931F9300910A0210910B0275
:100FA00020910C0230910D02602771278227932730
:100FB0000E9493071F910F9108950E948F07089533
:100FC0000E94DD0708950E94E00760930602709377
:100FD000070280930802909309020E943D0708953A
:100FE00060E070E0CB010E94E30708950F931F9328
:100FF00041E050E060E070E08A019B0104C0000F16
:10100000111F221F331F8A95D2F7C901B8010E9410
:10101000E3071F910F9108950F931F9341E050E054
:1010200060E070E004C0440F551F661F771F8A956B
:10103000D2F78091060290910702A0910802B09128
:1010400009028A019B01082B192B2A2B3B2BC90172
:10105000B8010E94E3071F910F9108950F931F930A
:1010600041E050E060E070E004C0440F551F661F8F
:10107000771F8A95D2F7CB01BA016095709580955C
:10108000909500910602109107022091080230917C
:10109000090260237123822393230E94E3071F9197
:1010A0000F9108950F931F9341E050E060E070E0CE
:1010B00004C0440F551F661F771F8A95D2F7809191
:1010C000060290910702A0910802B09109028A01DC
:1010D0009B01082719272A273B27C901B8010E942D
:1010E000E3071F910F9108950F931F93009106023C
:1010F000109107022091080230910902602B712B98
:10110000822B932B0E94E3071F910F9108950F9359
:101110001F9300910602109107022091080230915E
:10112000090260237123822393230E94E3071F9106
:101130000F9108950F931F930091060210910702DB
:101140002091080230910902602771278227932796
:101150000E94E3071F910F9108950895262F27708D
:1011600091E001C0990F2A95EAF723E076956795FB
:101170002A95E1F725E0269FF001279FF00D112425
:10118000E40FF51F50E040E0682F70E08191DF012F
:1011900011979B01042E02C0369527950A94E2F719
:1011A000217021952827292328272C934F5F5F4FF3
:1011B0004530510559F70895A82FA77023E096955B
:1011C00087952A95E1F725E0289FF001299FF00DEA
:1011D0001124E60FF71F50E040E080E0219130E05D
:1011E0000A2E02C0369527950A94E2F7217033271C
:1011F000042E01C0220F0A94EAF7822B4F5F5F4F43
:101200004530510559F70895262F953070F48F30E9
:1012100060F4682F70E08FE0989F600D711D1124BD
:1012200044ED51E0822F0E94AE080895292F953099
:1012300068F48F3058F490E064ED71E03FE0239F54
:10124000800D911D11240E94DC08089580E008950E
:10125000B0E0A0E0EEE2F9E00C94D72A8C01C09057
:101260000602D0900702E0900802F09009028091F7
:101270000A0290910B02A0910C02B0910D02C82AB3
:10128000D92AEA2AFB2ACFE1D0E0BC2ED701C60139
:101290000C2E04C0B695A795979587950A94D2F71A
:1012A00080FD09C0219788F7B12C8B2DCDB7DEB713
:1012B000E9E00C94F32AB8018C2F0E94D30F019718
:1012C00089F3F3CFCF93DF93EC010E942809BE018D
:1012D0000E94D30FDF91CF9108951F93CF93DF9397
:1012E000EB019091D301992339F0CB010E9462095F
:1012F000DF91CF911F910895882369F0CB010E945F
:101300002809182F682FCE010E940409BE01812FE1
:101310000E94D30FEDCFCB010E941609182FF6CFF4
:101320001F93CF93DF93C0910E0216E080910F02BE
:101330008C1304C0DF91CF911F910895D0E01C9FC2
:10134000F0011D9FF00D1124E05FFD4F40815181A0
:1013500062817381848195810E9485072196C7707F
:10136000E5CF40914002509141026091420270915C
:10137000430280914402909145020E94850708959E
:101380001F93CF93DF9380914502807F09F049C07E
:1013900080914202882309F444C080910E02C091DA
:1013A0000F026091400270914102A0914302B091FE
:1013B0004402D62FD72316E0C81799F190E0109772
:1013C00011F0DF3F19F401968770F6CF189F900156
:1013D000199F300D1124F901E05FFD4F4181471342
:1013E000F2CF40814613EFCF42814111ECCF4381D0
:1013F00054814A1B5B0B483C510528F780914502FC
:101400008F70806180934502F901EB5EFD4F808112
:101410008F708061808380E492E00E9413070E94B5
:101420009009DF91CF911F910895A1E1B0E0EBE128
:10143000FAE00C94D62A8C0185E0F801DE011D96B5
:1014400001900D928A95E1F7F801E28080E4C82EC0
:1014500082E0D82E609143027091440261157105BB
:1014600009F44EC19091400220914102892F8223BC
:101470008F3F09F445C140815181A380B480F09031
:101480004202F501E61BF70BFF2009F4EAC0809148
:101490004502382F307FE83CF10508F0A3C0311138
:1014A0006DC0FE2C251316C0941314C0E11012C099
:1014B0008F708061809345020E94B109C6010E942D
:1014C000130780914502F80185838F2D6196EAE02C
:1014D0000C94F22AA114B10429F0842F85238F3FA4
:1014E00009F027C180E0F82FF170DF2E80FF3CC0AB
:1014F00080910E0220910F0236E0821315C04D87B5
:101500005E878D859E850E946209292F22952F7006
:101510002230F0F0243018F59F70F1F0F801958139
:10152000907FD1F4D12C1EC090E0389FF001399FFC
:10153000F00D1124E05FFD4F6181651306C06081ED
:10154000641303C06281E6120FC001968770D5CF85
:101550009F7011F0882331F3805E883018F3C80142
:101560000E941307FD2CB1CFEE2009F4AECF80917D
:101570004502816080934502F12CA7CF251306C058
:10158000941304C0F801EE2009F487C0C8010E943A
:101590007307882319F1EE2009F18091450280320A
:1015A00070F0209140023091410238872F831986D4
:1015B000BB86AA868C87CE0107960E94130786E019
:1015C000F801A0E4B2E001900D928A95E1F70E9443
:1015D000C0090E94B109FF24F39477CFC8010E948B
:1015E0001307F9CF311113C07A2DB98AA88A6E2D4D
:1015F00089890E947B0780E492E00E94130786E0BD
:10160000F60111928A95E9F70E94B109B5CF251329
:101610000FC094130DC0E1100BC0F8018583C80101
:101620000E94130786E0F60111928A95E9F74DCFE3
:10163000C8010E947307882389F2EE2079F2809115
:101640004502803208F4BBCF209140023091410224
:101650003A8329831B82BD82AC828E83CE010196A0
:10166000ACCFE83CF10508F03EC0FE2CEE2009F4BA
:10167000B5CF25132AC0941328C08091450280FD60
:101680001BC0982F907FC1F0F8018583903F31F007
:10169000982F907F905F8F70892B8583C8010E945F
:1016A000130786E0F801A0E4B2E001900D928A955C
:1016B000E1F70E94B10909CF86E0F801A0E4B2E0A9
:1016C00001900D928A95E1F700CFC8010E9473073F
:1016D000811175CF80914502816080934502C801D8
:1016E0000E941307F2CE7A2DB98AA88A6E2D8989B5
:1016F0000E947B0786E0F60111928A95E9F7D9CF1F
:10170000EE2009F46BCFC8010E947307F82E8823DE
:1017100009F464CF86E0F801A0E4B2E001900D92F4
:101720008A95E1F780E492E00E9435040E94C009A6
:10173000C0CF81E08E25D7CEACE0B0E0E2EAFBE09E
:101740000C94DD2A4F83588769877A878B879C871B
:10175000CE0107960E94150A882369F08A859B8529
:10176000892B39F04F815885842F85238F3F09F0CD
:101770006BC016E05FC086E0FE013796DE01119671
:1017800001900D928A95E1F78A859B85892B89F3D3
:1017900088859F8189238F3F61F320910F0230E07C
:1017A000C90101968770992740910E0248171906C2
:1017B00071F40E94530710920F0210920E0286E0FD
:1017C000E0E4F2E0DF011D928A95E9F7D2CF96E0DE
:1017D000929FD001939FB00D1124A05FBD4FFE01D9
:1017E000319601900D929A95E1F780930F020E9435
:1017F0009009BFCF819FC0011124805F9D4F0E943F
:10180000150A8823E9F0E0910E021E9FF0011124D1
:10181000E05FFD4F408151816281738184819581B8
:101820000E94850780910E0290E0019687709927AB
:1018300080930E0280910E0290910F028913DACFED
:101840002C96E3E00C94F92A69857A858B859C8532
:101850000E9485078ECF682F809104019091050129
:101860000E94FB210895682F809104019091050149
:101870000E940922089580910401909105010E941F
:10188000172208958091660285958595859508951E
:10189000809166028770089590916602977081E04A
:1018A00009F480E008958091890208959091890259
:1018B000892B8093890208958095909189029823BD
:1018C0009093890208951092890208959091880258
:1018D000892B80938802089580959091880298239F
:1018E000909388020895109288020895809167026B
:1018F000089508950E94790C089590917D0492FFB7
:1019000008C090916702981721F0809367020E94A7
:101910007A0C089580916702882329F0109267025B
:1019200080E00E947A0C0895CF93DF93E091040148
:10193000F0910501809189028083E0910401F0918A
:101940000501808190918802892B808390916702A4
:10195000992381F0E0910401F09105018081892BA8
:10196000808380910401909105010E94672181117B
:101970000E948A0CC0910401D091050140E250E020
:1019800066E472E0CE010E946E2B892B59F080E252
:10199000FE01A6E4B2E001900D928A95E1F7CE0136
:1019A0000E941321DF91CF91089508950E94D50CD4
:1019B000089590917D0492FF11C098E0899F900155
:1019C0001124622B609366020E940C0880916602CB
:1019D0008595859585950E94D60C08950E940C08E2
:1019E00008951092660280E00E94D60C08959091AE
:1019F00066028095892380936602282F277091F4D0
:101A0000282F082E000C330B9217130659F09091D3
:101A10007D0492FF07C08595859585950E942E08C7
:101A20000E94F10C089590917D0492FB222720F9E9
:101A3000281769F080FB92F990937D0480917C04D3
:101A400090917D040E94640D82E00E94F70C08953D
:101A500080917D0482FB882780F991E089270E948C
:101A6000130D089581E00E94130D089580E00E94F7
:101A7000130D08956FEF7FEF90E080E00E94AD2B93
:101A8000089590E080E00E94892B21E0883E9E4FDF
:101A900009F020E0822F089582E090E00E947B2BE5
:101AA000089583E090E00E947B2B0895CF9384E01B
:101AB00090E00E947B2BC82F82E290E00E947B2B5B
:101AC000982F8C2FCF910895CF93C92F682F84E042
:101AD00090E00E948F2B6C2F82E290E00E948F2B6F
:101AE000CF910895AB01BC018FE090E00E94A12B43
:101AF0000895AB01BC0183E190E00E94A12B089501
:101B000060E070E0CB010E94790D089560E070E024
:101B1000CB010E94720D0E94800D089568EE7EEF49
:101B200090E080E00E94AD2B60E082E090E00E94B7
:101B30008F2B60E083E090E00E948F2B10920A02CE
:101B400010920B0210920C0210920D0260E084E0E1
:101B500090E00E948F2B64E082E290E00E948F2B45
:101B600060E085E090E00E948F2B60E086E090E0EE
:101B70000E948F2B6FEF87E090E00E948F2B40E058
:101B800050E0BA0188E090E00E94A12B60E08DE077
:101B900090E00E948F2B40E050E0BA0188E190E095
:101BA0000E94A12B60E087E190E00E948F2B40E033
:101BB00050E0BA018CE190E00E94A12B70E060E05F
:101BC00080E290E00E94AD2B40E050E0BA0188E155
:101BD00090E00E94A12B0E94860D08950E948E0D18
:101BE0000895682F8EE090E00E948F2B08950E9448
:101BF000E522609398027093990280939A029093E1
:101C00009B02609394027093950280939602909346
:101C100097020895089508950E940B0E089508955F
:101C20000E940F0E089582EB90E10E94FC200E941A
:101C30000A0E0E940C0E089581E008950E941C0E69
:101C40000895089508950E94210E0E94220E08957D
:101C50000E94D1100E94E0030E94A21E08950E94DB
:101C6000D0220E94C4110E94280E0E94F21C0E94E1
:101C7000151B0E94100E0895AAE0B0E0E2E4FEE019
:101C80000C94D12A0E94DA11A82E81110E94F70D1E
:101C90003AE8832E32E0932E10E000E0502E802FA1
:101CA0000E94FE106C01F401619071904F01681662
:101CB000790609F443C080919C0281FD0E940711BE
:101CC000B12CEE24E394F12C6C247D24C3018E21ED
:101CD0009F21892B69F10E941E0E8823B1F0BE82DC
:101CE0005F82CE20DF2081E0C114D10409F480E0BE
:101CF00088870E94D9228160782F9A8789874E81B0
:101D00005F8168858A850E940004000F111FF80119
:101D1000E657FD4F80819181E826F926F182E08225
:101D200081E0A11001C080E02A96EFE00C94ED2A3A
:101D3000B394EE0CFF1CFFE0BF12C8CF0F5F1F4F24
:101D40000530110509F0AACF8FEF89838A831B82A2
:101D50000E94D9228160782F9D838C8349815A818A
:101D60006B818D810E940004DBCF0E943C0E0E949B
:101D70005B1B0E94A11E0E94E9130E94F5030895B7
:101D8000CF93DF930E94D80FEC01811521E59207D4
:101D900008F042C0811530E5930708F09DC0883EE9
:101DA000910530F5803E910508F092C0883A910582
:101DB00088F4853A910508F084C08130910509F4D2
:101DC00087C0009709F484C0049708F081C0D0E070
:101DD000C0E07EC08F3B9105D0F7C85AD0E0CC0F51
:101DE000DD1FC15ADE4F0990D881C02DD46470C068
:101DF0008115904250F4C11581E0D80708F068C001
:101E0000CD3ED10520F3D06563C0C11590E4D9075C
:101E1000F0F2DF70D06A5CC0811525E5920700F50D
:101E2000811534E5930708F08BC0811543E59407CD
:101E300008F073C0C11582E5D80708F469C0CE0167
:101E40008370992721E030E002C0220F331F8A956A
:101E5000E2F7C695C69580E2C89FE001112454C000
:101E6000C11599E5D907A8F4C11528E5D20708F0EE
:101E70006CC0C11536E5D30708F0A9CF8C2F0E949E
:101E80006F10C82FD0E0DC2FCC27CC27DF71D062B9
:101E90001FC0C1154AE5D40708F45CC0CE019056B6
:101EA0008115904208F093CF8D2F8F710E946F1093
:101EB00090E0982F882788279F719C012C2BE9019F
:101EC000E6CFC55AD0E0C357DE4FC881D0E0D0641A
:101ED000CE01DF91CF910895E4E096958795EA953C
:101EE000E1F783702C2F26952695237040E2249FDE
:101EF00090011124382B8C2F8370C1E0D0E002C0F8
:101F0000CC0FDD1F8A95E2F7C22BD32BDC68E0CF24
:101F1000DC2FCC27C16FD06ADBCF8370992721E0FB
:101F200030E002C0220F331F8A95E2F7C695C695AE
:101F300090E2C99FE0011124C22BD32BDA68C8CFED
:101F4000D82FCC27C46FD06AC3CFDC2FCC27C06F6B
:101F5000D06ABECF8C2F8F700E946F1034E0D69560
:101F6000C7953A95E1F7CF709C2FEC01D069B0CFBF
:101F7000972F7530A8F46F3098F470E02FE0929F9F
:101F8000600D711D1124FB019BE4899FE00DF11D83
:101F90001124EE0FFF1FE455FF4F85919491089592
:101FA00080E090E008950E94B80F0E94C00E08954E
:101FB00082389105B1F1B0F48133910509F475C00F
:101FC00048F48932910509F469C08A32910509F40F
:101FD00073C008958533910509F459C0893391057B
:101FE00001F10895833E9105A9F138F4803E9105F1
:101FF000F9F0823E910549F10895863E9105A9F1D7
:10200000873E9105C9F1843E910519F520917D0423
:1020100021FF1FC080917C0484FD14C087EE90E0F6
:10202000089520917C042370A1F080EE90E0089543
:1020300020917C0420FD47C030917D0430FF09C011
:1020400024FF44C090E080E004C020917C0422FD85
:10205000F7CF089520917C0422FD3BC030917D0490
:1020600030FDE3CF24FFF5CFEDCF20917C0423FF9B
:10207000F0CF24FDE7CFD2CF20917C0423FD2CC0EC
:1020800030917D0431FFEECF84EE90E008952091F1
:102090007C0425FFDECF89E290E0089520917C0446
:1020A00025FFD7CF85E390E0089520917C0426FF9B
:1020B000D0CF8AE290E0089520917C0426FFC9CF1A
:1020C00081E390E0089589E390E0089583EE90E045
:1020D000089582EE90E0089586EE90E00895909144
:1020E0007C0492FF06C0282F28712830F9F4877FDE
:1020F000846093FF06C0282F28712831F1F4877E71
:10210000846120917D0420FF06C0382F387138305B
:10211000D9F4877F816021FF06C0282F28712831DC
:10212000D1F4877E816194FD877E0895282F2471E4
:102130002430F9F68B7F8860DCCF282F247124317E
:1021400001F78B7E8861DDCF382F3171313019F77F
:102150008E7F8860E0CF282F2171213121F78E7E7C
:102160008861E1CF80E008950E943A0D08950E94B1
:10217000DA112FEF86E791E0215080409040E1F79F
:1021800000C000000E94DA1180E00E94FE1080FF73
:1021900004C00E94B4100E94242308950E94B71026
:1021A00008950E94410D811102C00E94EE0D0E940F
:1021B0004C0D80939C020E94560D90937D04809359
:1021C0007C040E94CE100E94510D682F70E090E0B8
:1021D00080E00E94A1076091060270910702809141
:1021E0000802909109020E94E007089508950E9454
:1021F000F610089508950E94FA100895E82FF0E06F
:10220000EE0FFF1FE857FB4F8081918108950895DD
:1022100080EA8A95F1F7089500C008950E94081198
:102220000895F894E82FE295EF70F0E031A1282F9F
:102230002F7081E090E001C0880F2A95EAF7982F6F
:102240009095932391A392A1892B82A378940895CA
:102250000F931F93CF93DF93C0E9D1E089918F3F14
:1022600011F00E94111181E0CF39D807B9F7CFE9F9
:10227000D1E004EA11E089918F3F11F00E94111121
:102280000C171D07C1F7DF91CF911F910F91089592
:102290008F929F92BF92CF92DF92EF92FF920F9315
:1022A0001F93CF93DF93D82EE92EF62E8A01C62FE7
:1022B000D0E0C057DE4F28812F3F09F453C0F89477
:1022C000E22FE295EF70F0E031A12F7081E090E015
:1022D00001C0880F2A95EAF7932F982B91A392A11A
:1022E0008095892382A378940E940C118FE9882E0F
:1022F00081E0982EED2DFE2DBF01665F7F4FE12C12
:102300006801C094D094D401BD904D018191919108
:10231000AF0142505109BFEFBB1681F12B2D229521
:102320002F7030E0D90190962C9130E0BB2DBF701A
:1023300002C035952795BA95E2F720FD1FC0802B86
:10234000912BDA018D939C93EE24E3946E177F0713
:10235000D1F688818F3F11F00E9411116E2D8F2DC3
:102360000E940E11DF91CF911F910F91FF90EF907E
:10237000DF90CF90BF909F908F9008958C219D21EA
:10238000DA018D939C93E2CF0E9428118AE0E8E85D
:10239000F4E0DF01982F1D929A95E9F7EEE7F4E05B
:1023A000DF011D928A95E9F785E00E942F120E94B5
:1023B0003B030895CF92DF92FF920F931F93CF9329
:1023C000DF93CDB7DEB72A970FB6F894DEBF0FBE06
:1023D000CDBF8E010F5F1F4F8AE0F80111928A95E1
:1023E000E9F7F12CCC24C394D12CA6016F2DC801A0
:1023F0000E944811F394CC0CDD1CFFE0FF12F5CFD6
:102400004AE050E0B8018EE794E00E946E2BFF2472
:10241000F394009709F4F12C892B41F08AE0F8013C
:10242000AEE7B4E001900D928A95E1F72F2D45E0DB
:1024300068E874E08EE794E00E9430120E943E0348
:102440008F2D2A960FB6F894DEBF0FBECDBFDF9159
:10245000CF911F910F91FF90DF90CF900895089535
:10246000FF920F931F93CF93DF93F82E092F162F10
:10247000D72FC42F222349F081E080939F020E942E
:10248000D92290939E0280939D0280919F0288237F
:10249000A1F080919D0290919E020E94F1220597E9
:1024A00060F0EF2DF02FA12FBD2F90E080E0D0E065
:1024B0008C179D073CF010929F02CDB7DEB7E5E088
:1024C0000C94F72A219131912D933D930196F0CFF1
:1024D0000E94FE240E942F0E0E940B2508950E9448
:1024E00010250E94B50E0E942A2508950E9472228E
:1024F0000E94E4240E94130E0E9468120E946F1230
:102500000E94230EFBCF8091A60280FF0DC0609138
:102510000B0170E0660F771F6038710570F561156B
:10252000710569F1862F089581FF07C060910B0145
:1025300084E0689FB0011124EFCF60910B0182FD10
:102540000AC08091A5028823A9F020910A01609118
:102550000B01821710F088E0ECCF869FC001112498
:1025600033E0880F991F3A95E1F7622F70E00E94DF
:10257000612AD2CF68E070E0D5CF8FE7089581E07F
:1025800008958091A60280FF0CC06091070170E061
:1025900075956795759567956115710549F1862F54
:1025A000089581FF06C06091070170E075956795F9
:1025B000F3CF6091070182FD0BC09091A402992393
:1025C000A1F06091060180910701961738F0682FFD
:1025D00070E06038710500F38FE70895899FC001AE
:1025E000112470E00E94612AF4CF61E070E0D7CF3F
:1025F00081E008958D3E31F40E948312819580938D
:10260000AA0208958E3E19F40E948312F8CF8F3EDD
:1026100031F40E94831281958093A9020895803F2E
:1026200019F40E948312F8CF893F29F40E94C11245
:102630008093AB0208958A3F21F40E94C1128195D4
:10264000F7CF8B3F31F40E94C11281958093AC0289
:1026500008958C3F19F40E94C112F8CF9FE0980FA3
:10266000983070F4815F990B21E030E001C0220FB7
:102670008A95EAF78091A802822B8093A802089598
:102680008D3F31F48091A60281608093A602089567
:102690008E3F21F48091A6028260F7CF8F3FB9F779
:1026A0008091A6028460F1CF4091A9028D3E59F439
:1026B0008091AA0287FF0DC01092AA0241110BC09F
:1026C0001092A50208C08E3E81F48091AA021816CD
:1026D0009CF3442381F08091AB029091AC02892B52
:1026E00009F05AC01092A40208958F3E49F447FFA2
:1026F000F0CF1092A9028091AA028111ECCFE0CF15
:10270000803F19F41416ACF3E4CF9091AB02893FEB
:1027100029F41916F4F61092AB02DBCF8A3F19F4B4
:1027200097FFD7CFF8CF9091AC028B3F29F497FF5A
:10273000D0CF1092AC02CDCF8C3F19F41916CCF348
:10274000C8CF9FE0980F983090F4815F990B21E0FB
:1027500030E0B90102C0660F771F8A95E2F7CB011E
:1027600080959091A80289238093A802B2CF8D3FD3
:1027700031F48091A6028E7F8093A602AACF8E3F6D
:1027800021F48091A6028D7FF7CF8F3F09F0A1CF72
:102790008091A6028B7FF0CF08950E94D9229C01E0
:1027A0009091A9028091AA02982B21F03093A30264
:1027B0002093A2029091AB028091AC02982B21F061
:1027C0003093A1022093A00287EA92E00E942D217B
:1027D0000895A6E0B0E0EFEEF3E10C94DD2A86E088
:1027E000E7EAF2E0DE01119601900D928A95E1F799
:1027F0001092A9021092AA021092AB021092AC029F
:102800008B819C81892B81F08091A2029091A302FF
:102810000E94F122AC019091A502992391F180913F
:102820000C0184171506D0F18D819E81892B91F0C2
:102830008091A0029091A1020E94F122AC0190919E
:10284000A402992309F46BC080910801841715062E
:1028500008F473C0BE016F5F7F4F87EA92E00E9469
:10286000292281110E94CD1386E0FE013196A7EA4C
:10287000B2E001900D928A95E1F72696E3E00C9480
:10288000F92A20910D018AE0289F90011124241734
:10289000350750F69F5F9093A50202C09F3FD1F786
:1028A0001B81112359F00E9483129FEF11160CF423
:1028B00091E0899F802D11248093A9021C8111230E
:1028C00059F00E9483129FEF11160CF491E0899F3A
:1028D000802D11248093AA023091A902332309F498
:1028E000A3CF2091AA02222309F49ECF45EB340303
:1028F000C0011124992359F09093A90245EB2403B8
:1029000090011124332339F03093AA028DCF81E056
:102910008093A902F3CF81E08093AA0285CF209112
:1029200009018AE0289F900111242417350708F037
:1029300091CF9F5F9093A40202C09F3FD1F71D816A
:10294000112359F00E94C1129FEF11160CF491E06F
:10295000899F802D11248093AB021E81112359F091
:102960000E94C1129FEF11160CF491E0899F802DF7
:1029700011248093AC023091AB02332309F46ACF67
:102980002091AC02222309F465CF45EB3403C0014A
:102990001124992359F09093AB0245EB2403900145
:1029A0001124332339F03093AC0254CF81E080936B
:1029B000AB02F3CF81E08093AC024CCF86E0E7EA34
:1029C000F2E0DF011D928A95E9F71092A5021092BC
:1029D000A4021092A6020895EF92FF920F931F9304
:1029E000CF93DF93EB01E82FD1110EC0442321F0E8
:1029F000F0E0EE50FD4FE4916E2F7E2F8E2FCDB77D
:102A0000DEB7E6E00C94F62A0D2F10E0282F30E018
:102A1000442329F02E503D4FF901249130E0F6E097
:102A2000CF9FC0011124EFEFF0E0BF010E944D2ABB
:102A3000AB018C2F90E0880F991FA5E5A49FB001F2
:102A4000A59F700D1124861B970B982F990F980F37
:102A5000BF01601B710B629FD001639FB00D729F1D
:102A6000B00D11248B2F9D9FB0011124672F772764
:102A7000EF01C61BD70BBE01629FE001639FD00D23
:102A8000729FD00D11247F01E91AF108E09EB00178
:102A9000E19E700DF09E700D1124672F7727E61BC5
:102AA000F70BE29F8001E39F100DF29F100D1124A0
:102AB000E12F722F4230510599F048F4411551052C
:102AC00069F04130510581F0EB2F8D2F07C0443064
:102AD000510569F080F046305105B1F76E2F8FCF68
:102AE000E22F7B2F812FFACFE22F7D2FF7CFEB2F15
:102AF000822F712FF3CF7B2F822FED2FEFCF41E06D
:102B00000E94EC14089508950E947F150895CF93B4
:102B1000DF93762FE901682F842F0E948415798333
:102B200068838A83DF91CF910895413A08F040EAA3
:102B30000E948715089580919204982F9E7F61F4DA
:102B4000817082608093920480919504813A18F09C
:102B500080EA8093950408958635B0F3817084658A
:102B6000F1CF88E090E00E94832B0895CF92DF920E
:102B7000EF92FF926B017C010E949B15B701A601A9
:102B800088E090E00E94A12BFF90EF90DF90CF9023
:102B90000895E2E9F4E083E0808311828FEF82837D
:102BA00080EA8383148260817181828193810E9493
:102BB000B61508958091920480FF02C0869508950D
:102BC00080E0089590919604933018F49F5F90935D
:102BD0009604882351F0609192047091930480913F
:102BE0009404909195040E94B615089581E00E9486
:102BF000E215089590919604992319F091509093BD
:102C00009604882351F0609192047091930480910E
:102C10009404909195040E94B615089581E00E9455
:102C2000FA15089570E00E94B31E08956091120194
:102C30008091920480FF0BC08091110123E0829F5C
:102C4000C001112489569B4F0E941216089580914D
:102C500013019091140123E0829FF0011124E956A1
:102C6000FB4F891748F71182108212828F5F3396CB
:102C7000F8CF9091920490FF0EC090911301209193
:102C8000140133E0939FF0011124E956FB4F921792
:102C900018F00E94161608958183608342839F5F17
:102CA0003396F5CFA3E0B0E0E8E5F6E10C94DE2A38
:102CB0009091920490FF0AC09E012F5F3F4F0E94A7
:102CC00095154B8169818A810E9439162396E2E02D
:102CD0000C94FA2ACF93DF93EC01EC81F0E0E351FE
:102CE000FE4F4491E2E9F4E0628181810E94521634
:102CF0008C818F5F8C83DF91CF910895CF93DF9389
:102D0000EC01E2E9F4E0438162818C810E94521679
:102D10008C818F5F8C83DF91CF910895A3E0B0E029
:102D2000E4E9F6E10C94DC2A8C018091AD0281117A
:102D30000AC09E012F5F3F4F40EA6FEF0E9495153A
:102D40008A818093AD02F8016481613069F08091DD
:102D5000AD0240E0662361F040E0623011F4409142
:102D6000AD0280E060E004C06091AD0240E080E030
:102D70000E943916F801848190E0019663E070E0CA
:102D80000E94612A84832396E4E00C94F82AA3E04D
:102D9000B0E0EDECF6E10C94D72A082FD62EE42E05
:102DA000C22E9091920490FF29C0E92FE695AE2F94
:102DB000B0E0AC55BE4F8C91809349049E7F923019
:102DC00009F59E012F5F3F4F802F0E9495154B8183
:102DD00069818A810E94391600939304D0929404E9
:102DE000E0929504CC2051F060919204709193048C
:102DF00080919404909195040E94B6152396E9E081
:102E00000C94F32A823019F4E0909504E5CF8630D3
:102E100019F400919304E0CF8930D9F38931E1F6B8
:102E2000E9516E2F6170B62EE695F0E0E351FD4F4B
:102E30001491F12C60911501F61618F00E941616E7
:102E4000CBCFF19EC001112470E00E944D2A802F4B
:102E5000B11014C0860F20911301622F6F0D7727D8
:102E6000771F9B01220F331F260F371F29563B4F19
:102E70004E2D6D2D0E949515F394DCCF861BEBCF64
:102E8000E2E9F4E09181282F4381628188E0890F93
:102E90000E94C716089581E00E9440170895E2E954
:102EA000F4E09181282F4381628188EF890F0E948D
:102EB000C716089581E00E944F170895E2E9F4E0F3
:102EC000628128E0620F08F46FEF282F438181812F
:102ED0000E94C716089581E00E945E170895E2E9F6
:102EE000F4E0628128E0621B08F460E0282F43814F
:102EF00081810E94C716089581E00E946F1708958E
:102F0000E2E9F4E0438128E0420F08F44FEF282F74
:102F1000628181810E94C716089581E00E94801716
:102F20000895E2E9F4E0438128E0421B08F440E020
:102F3000282F628181810E94C716089581E00E9436
:102F40009117089520E00E94C7160895EF92FF920E
:102F50001F93CF93DF93EC0110E0EE24EA94F12C61
:102F600060911501161770F00E9416169A818C81D7
:102F700090FF27C08F5F8C83DF91CF911F91FF90CF
:102F8000EF90089520911301422F410F5527551FAF
:102F9000CA019A01220F331F280F391F29563B4FB0
:102FA00070E0C7010E94612A962F8C8140919504A0
:102FB00060919404199F800D11240E9495151F5F44
:102FC000CFCF8150D8CFB0E0A0E0E9EEF7E10C948C
:102FD000D62AFC0182810FEF80FF01E010E040E57E
:102FE000A42E80911501181798F00E941616809152
:102FF000AF02013009F04FC0811102C0809115016C
:1030000081508093AF02CDB7DEB7EAE00C94F22A8C
:10301000C0911301C12ED12CCC0DDD2DD11DCE01BF
:10302000880F991FC80FD91FC956DB4F1982188204
:103030001A8234E0E32EF12CB12C8091AF028B0D7B
:1030400081351CF16A2D0E943F2A892F082E000C21
:10305000990BC816D90691F4809195048E9DA00114
:103060008F9D500D112455954795559547959E0177
:1030700060919404809193040E949515B00EF1E044
:10308000EF1AF108D1F61F5FACCF87FFDFCF909129
:103090001501890FDBCF90E001966091150170E07A
:1030A0000E94612AAECF0F931F93CF93DF9380913D
:1030B00013019091140123E0829FF0011124E9563D
:1030C000FB4F891740F1C0E0D3E060911501C617AE
:1030D00040F10E94161620910F018091AE02820FDE
:1030E0008093AE0290911001920F909310011916E7
:1030F00054F4082E000C990B409115014150550BCA
:10310000841795071CF0219520930F01DF91CF9133
:103110001F910F9108951182108212828F5F339652
:10312000D0CF0C2F10E070E0C8010E94612A2091DE
:103130001301820F482F50E02091AE02022E000CA6
:10314000330B02171307BCF020911001022E000C64
:10315000330B201731077CF08D9F900111242956E5
:103160003B4F4091950460919404809193040E9498
:103170009515CF5FAACFFA01EE0FFF1FE40FF51FE1
:10318000E956FB4F118210821282F3CFB0E0A0E02B
:10319000ECECF8E10C94D42AEC014C81042F10E003
:1031A0009801D8010E94A52A9B01AC010E94BB2A6C
:1031B0004B015C01E0E2F0E0E01BF10BA5E5B0E0C3
:1031C000AC019B010E94BB2A6B017C019F01DF01C6
:1031D0000E949D2A9B01AC010E94C62A9B01AC0162
:1031E000280D391D4A1D5B1DC701B6010E94752AB5
:1031F000F22E822F90E039E23F1520F143E0249F28
:103200009001112435952795122F109500E085E542
:10321000E82EEF1880911501081718F10E94161674
:103220009C8181E0992319F0903219F48FEF8093FB
:103230000E0180910E01890F8C83CDB7DEB7ECE0D3
:103240000C94F02A25E530E0B901681B790B9B014D
:10325000220F331F260F371F37FFD4CF2F5F3F4F6B
:10326000D1CF8E2D01FD8F2D20911301622F600F84
:103270007727771F9B01220F331F260F371F2956F1
:103280003B4F412F609194040E9495150F5FC2CF70
:103290000F931F93CF93DF93EC0110E000E0909128
:1032A00015019017110609F06CF40E9416168C8116
:1032B00090E00196817099278C83DF91CF911F91C7
:1032C0000F91089520911301A801420F511D9A01F9
:1032D000220F331F240F351F29563B4F4C8160911D
:1032E00094048091930496959017110651F04CF038
:1032F000442349F0409195040E9495150F5F1F4F9C
:10330000CECF4423B9F340E0F7CFB0E0A0E0EBE844
:10331000F9E10C94D02AFC016280448081E084832E
:10332000EDEEF1E07490ECE6F2E0E491812C75E0D2
:10333000972EF2E0CF2EDD24D394AA24AA94B12CA8
:1033400055245A94E7190E2F10E080911501881624
:1033500038F00E941616CDB7DEB7E0E10C94EC2AE7
:10336000E82CF12C82E0861568F09E9CF0019F9C71
:10337000F00D1124E055FD4F8091930480838091DE
:1033800094048183411023C09E9CF0019F9CF00D0A
:103390001124E055FD4F1382128220911301C701C1
:1033A000820F911D9C01220F331F280F391F2956B0
:1033B0003B4F9E9CF0019F9CF00D1124E055FD4F6A
:1033C0004281618180810E9495158394BECF9E9C2D
:1033D000E0019F9CD00D1124C055DD4F8B818823C7
:1033E000E9F081508B83859DC00111246C8170E0D0
:1033F0000E944D2AFB01FF27E351FE4F8491E82FE5
:10340000E719E59DC0011124B8010E944D2A809161
:103410009504689FB00111247A83BFCF0E94512B7D
:1034200020919504269521582C9DA0012D9D500D8D
:103430001124452F5527841795070CF0AECF82E055
:10344000861588F40E94512BB5010E94612A888359
:103450000E94512B209194042695622F70E00E94C7
:10346000612A280F29839E9CF0019F9CF00D112456
:10347000E055FD4F128280919504893C58F088EC0C
:103480009E9CF0019F9CF00D1124E055FD4F84831C
:10349000838383CF8431A0F784E1F2CFE2E9F4E0C3
:1034A00080818E7F808360817181828193810E947F
:1034B000B61510924A042FEF80E792E02150804029
:1034C0009040E1F700C000000E9416160895E2E95E
:1034D000F4E080818E7F808310924A042FEF80E792
:1034E00092E0215080409040E1F700C000000E942F
:1034F0001616089510924A048091470481110AC05B
:1035000081E0809347048091920481708093460407
:103510000E94671A089560919204669570E04BE0EE
:1035200050E086E191E00E94612B892B19F481E043
:1035300080934A040E94D9229093410480934004CE
:1035400008959091920490FF2BC09170811129C031
:10355000926090939204662351F06091920470916E
:10356000930480919404909195040E94B615609103
:103570009204669570E04BE050E086E191E00E9495
:10358000612B892BA9F010924A0481E080934304B7
:103590004091950460919404809193040E94A21735
:1035A00008958B3210F09465D4CF880F982BD1CF2B
:1035B0000E948B1AEACF682F90919204969581E031
:1035C000890F8B3208F081E00E94A11A089581E0F2
:1035D0000E94DB1A0895682F9091920496958FEFC0
:1035E000890F09F48AE20E94A11A089581E00E94DD
:1035F000EB1A089561E00E94A11A0895E2E9F4E04F
:1036000080818160808386950E94FA1A0895809156
:10361000920480FF03C00E944E1A08950E94FE1A71
:10362000089560E00E94A11A0895809148048111D4
:103630002EC00E94410D811104C00E94EE0D0E9417
:10364000C9150E94B11560939204709393048093FE
:103650009404909395046E7F61F40E94C9150E94B2
:10366000B1156093920470939304809394049093A3
:1036700095040E949B1510924A048091920480FF49
:1036800003C086950E94111B81E080934804089531
:10369000E2E9F4E080818160808386950E94111BBD
:1036A0000895109247048091460481110E94481B9E
:1036B0000E948B1A08950F931F93CF93DF938091ED
:1036C0004A048823B9F180914904E0919204E69577
:1036D000E81BE0934204823091F5F0E0E751FE4FA1
:1036E000E491CE2FD0E00AE616E1809143048823CE
:1036F00061F0109243040E94D92290934104809378
:10370000400410924504109244040E94D922E09192
:103710004004F09141048E1B9F0B8F3F9F4750F454
:10372000EC0FFD1FF0934104E093400480E494E02B
:10373000F8010995DF91CF911F910F91089586307F
:1037400049F4F0E0EA51FE4FE491CE2FD0E00EE7CD
:1037500016E1CBCF893051F4E695F0E0ED51FE4F04
:10376000E491CE2FD0E006EA17E1BFCF8F3051F4BD
:10377000E695F0E0E052FE4FE491CE2FD0E003EE6C
:1037800017E1B3CF853149F4F0E0E352FE4FE49105
:10379000CE2FD0E003E518E1A8CFC8E2D0E006ECD8
:1037A00018E1883109F4A1CF833239F4EBEDF1E06F
:1037B000C591D4910EE816E198CFC4EFD1E008E4AA
:1037C00019E1843209F491CFC0EDD7E003E815E1A7
:1037D000853209F08ACF8E2F63E00E94332AE92FC9
:1037E000F0E0E852FE4FE491CE2FD0E005E819E179
:1037F0007CCFFA01811101C0FB0109950895CF9397
:10380000DF93C82FD62F0E94DA158C1748F00E943C
:10381000DA158D1728F40E94E71ADF91CF910895E9
:103820008C2F0E94FA1AF9CF1F93CF93DF93EC01EC
:10383000FB01128111111BC00E94530C8272CD3CFE
:10384000FCE5DF0709F4A0C008F045C0C73CECE583
:10385000DE0709F485C0F8F4C43C9CE5D90709F4F7
:1038600075C050F4C33CDC4509F46DC011E0812FF4
:10387000DF91CF911F910895C53C9CE5D90709F4CC
:103880006AC04AE557E16BE477E1C63CDC4571F775
:103890000E94F91BECCFCA3CFCE5DF0709F46AC0C3
:1038A00068F4C83CECE5DE0709F45FC04BE657E17D
:1038B0006CE777E1C93CDC4559F3D8CFCB3C9CE5BC
:1038C000D90709F45CC04EE056E166EF75E1CC3CE7
:1038D000DC45F1F2CBCFC23DFCE5DF0709F463C064
:1038E00098F4CF3C9CE5D90709F457C008F451C0BF
:1038F000C03DFCE5DF0709F453C0C13DDC4509F0DC
:10390000B5CF6EE089E01CC0C53D9CE5D90709F440
:1039100050C058F4C33DFCE5DF0709F447C0C43D7F
:10392000DC4509F0A3CF88E135C0C63D9CE5D90749
:1039300009F442C06AE285E2CE35DD4509F096CF52
:103940000E94FF1B94CF0E94071B91CF46EF5AE1C4
:1039500067EE7AE19DCF47EE5AE166EF7AE198CFC4
:103960004BE457E16AE577E193CF4CE757E16BE62B
:1039700077E18ECF4EE957E16DE877E189CF4DE8E9
:1039800057E16EE977E184CF46EF55E16EE076E1ED
:103990007FCF81E00E94FA1A6ACF65E082E0D0CF43
:1039A00068E086E0CDCF64E18FE0CACF67E185E1D2
:1039B000C7CF62E289E1C4CF83E2ECCF86E090E03A
:1039C0000E947B2B0895682F86E090E00E948F2B49
:1039D0000895E7E8F5E080818470896280830E9421
:1039E000E31C08950E94410D811104C00E94EE0D58
:1039F0000E94E91C0E94DE1C80938705803320F022
:103A0000877088628093870590918705892F8170E0
:103A100090FF04C0892F8695869586950E94FB1D90
:103A2000089580918705982F96959695969595304F
:103A300040F49F5F990F990F990F8770892B80939E
:103A40008705809187058160809387050E94E31C2C
:103A5000809187058695869586950E94FB1D089521
:103A600080918705982F987F79F0885080938705FB
:103A7000887F91E009F490E08091870590FB80F9C0
:103A8000809387050E94E31C809187058695869523
:103A900086950E94FB1D08958091870580FD13C0C7
:103AA000816080938705813019F489E080938705D0
:103AB000809187050E94E31C8091870586958695F5
:103AC00086950E94FB1D08958091870580FF08C0A0
:103AD0008E7F809387050E94E31C80E00E94FB1D7F
:103AE00008958091870580FF03C00E94641D08959A
:103AF0000E944C1D089590918705892F8695869583
:103B000086958F5F8F7197708630E0F4880F880FED
:103B1000880F892B8093870580918705887F91E0A6
:103B200009F490E08091870590FB80F980938705E8
:103B30000E94E31C809187058695869586950E9454
:103B4000FB1D089590938705E7CF863008F085E048
:103B5000909187059770282F220F220F220F922B0A
:103B600090938705987F21E009F420E090918705E4
:103B700020FB90F9909387050E94FB1D08950E94F9
:103B8000A51D809187050E94E31C08959C01FB01FF
:103B90008281882349F12E3BFCE53F07C9F040F4C0
:103BA0002C3BECE53E0769F02D3B3C4579F0089550
:103BB000203C9CE5390791F070F0213C3C4589F0B0
:103BC000089585E00E94BF1D80E0089580E0FACF4F
:103BD0000E94301DF9CF0E94111DF6CF0E94711D69
:103BE000F3CF0E947B1DF0CF81E00895269A2E9896
:103BF00008952E9808958F929F92AF92BF92EF9260
:103C0000FF920F931F93CF93DF93C82F8630C0F599
:103C1000811137C0809180008F7D809380000E9449
:103C2000F91DA0918600B09187002C2F30E00E94F2
:103C3000A52A25E030E040E050E00E94752A890185
:103C40009A0180918600909187006CE070E00E945C
:103C50004D2A60177107D8F0C80169E070E00E9432
:103C60004D2A70938B0060938A00DF91CF911F9152
:103C70000F91FF90EF90BF90AF909F908F9008951D
:103C8000C5E080918000806280938000CACF8091DF
:103C9000860090918700E0908600F0908700E09188
:103CA0008600F0918700C6E0D0E0BE010E944D2A58
:103CB000060F171F211D311D4801590185E0880C91
:103CC000991CAA1CBB1C8A95D1F7C701BE010E9492
:103CD0004D2A9F0150E040E0260F371F411D511D26
:103CE000C501B4010E94752A49015A01E09186007C
:103CF000F0918700CA01B9010E94232A9B01AC01FF
:103D0000DF010E94BB2A9B01AC01C501B4010E94E6
:103D1000232A2FE096958795779567952A95D1F771
:103D2000009186001091870030E020E00617170709
:103D30002807390708F095CF6091860070918700B9
:103D400090CF08950E94F61D82E28093800089E161
:103D5000809381008FEF9FEF909387008093860080
:103D60000E94F21C08956A9A4EB14B7F5EB1546076
:103D7000EFB7F8949B01220F331F260F371F280F30
:103D8000391F2817390741F4EFBF8FE594E00197F9
:103D9000F1F700C000000895DC016D91CD0178E0DD
:103DA0005EB9000000C067FF4EB9660F000000C09A
:103DB00000C000C04EB900C07A9591F7E2CFCF9312
:103DC000DF93EC01FB018281882309F433C1C43005
:103DD000FDE5DF07C0F5CB3F9CE5D90730F49E0138
:103DE00022503C4524313105B0F50E94560D909388
:103DF0007D0480937C04C1318CE5D80709F4EEC0C2
:103E000008F069C0C930ECE5DE0709F4D5C0C8F593
:103E1000C5308CE5D80709F4C7C000F5C330ECE520
:103E2000DE0709F4B9C008F0BBC0C230DC4509F4B4
:103E3000ADC080917C0490917D040E94640D0E942D
:103E4000530780E008C0C236EDE5DE0771F2C63ADE
:103E5000FDE5DF0751F2DF91CF91089580917C0459
:103E60008062C7309CE5D90709F493C080917C0437
:103E70008061C830DC4508F48CC080917C0480648B
:103E800088C080917C048B7FCD30FCE5DF0709F48E
:103E900080C098F480917C048E7FCB309CE5D9075C
:103EA00009F477C080917C048C60CC30DC4508F448
:103EB00070C080917C048D7F6CC080917C048F7E6B
:103EC000CF30FCE5DF0709F464C008F47BC08091C3
:103ED0007C048F7D5EC0CE3F9CE5D90709F47AC093
:103EE00050F5C531FCE5DF0709F486C098F48091F0
:103EF0007C04837FC3319CE5D90709F44AC008F4E8
:103F000071C00E94530790917C04892F97FB87F919
:103F100080583FC0CC3FFCE5DF0709F449C008F0FA
:103F200055C080917D048160CB3FDC4509F081CF95
:103F300080937D047ECFC230EDE5DE0709F468C0D2
:103F4000A8F4C1158DE5D80709F452C080917D040D
:103F50008360C130DD4560F380917D04982F90959A
:103F600091708E7F892B90FB81F9E2CFC236EDE50F
:103F7000DE0709F451C0C63AFDE5DF0709F453C076
:103F8000C330DD4509F055CF80E043C080917C040B
:103F9000816080937C044DCF80917C048260F9CF56
:103FA00080917C048460F5CF80917C048860F1CF9F
:103FB00080917D048260BCCF0E94530780917C0475
:103FC0008068E7CF80917C04877FE3CF80917D0478
:103FD0008E7FAECF80917D048D7FAACF80917C04AF
:103FE0008F7BD7CF0E94530780917C048F77D1CFEE
:103FF00080917D048C7F9CCF80917C0482FB9927EB
:1040000090F921E0922790FB82F990FB83F9C1CFD0
:1040100081E00E94F10D0DCF90917C04892F8F7E5D
:1040200094FF8061B6CF90917C04892F8E7F90FFA2
:104030008160AFCF81E00FCFCF93DF93EB0186316B
:104040009C4511F50E94530C9A81992399F08A7A24
:1040500091E009F490E090934B04811109C089E24A
:104060000E942B0C0E94940C80E0DF91CF91089568
:1040700085E3F6CF80914B04811104C089E20E9450
:10408000330CF0CF85E3FBCF81E0EFCF0F931F938D
:10409000CF93DF93C42FD22FFC0182818823C9F0F4
:1040A00040934E040E94D92290934D0480934C0477
:1040B00080E28C0F883040F4C77081E001C0880F27
:1040C000CA95EAF70E94DA04DF91CF911F910F9110
:1040D000089510914E04141332C080914C049091B5
:1040E0004D040E94F122883C910548F5C0E2CD0FB5
:1040F0001D17B9F080E2810F883040F4177081E01D
:1041000001C0880F1A95EAF70E94E104C83048F40C
:1041100081E09D2F977001C0880F9A95EAF70E9461
:10412000DA04802F0E94D104C83070F6D77081E085
:1041300001C0880FDA95EAF70E94E104C5CF80E25A
:104140008C0F883008F6C77081E001C0880FCA95CF
:10415000EAF7F2CF0F939C01CB01243F4CE53407E3
:1041600059F1A8F4293DFCE53F0701F12A3D4CE552
:104170003407D1F1283D3C4591F406E221EE41EEB1
:1041800068ED7CE50E94462080E00F910895263F6F
:10419000FCE53F07E9F0B0F0273F3C45F9F0FC01B2
:1041A0008281882339F110924E04EFCF07E225EE89
:1041B00045EE69ED7CE5E6CF06E221EE40EE64EFE8
:1041C0007CE5E0CF07E225EE44EE65EF7CE5DACF53
:1041D00006E221EE42EE66EF7CE5D4CF07E225EE63
:1041E00046EE67EF7CE5CECF08E221E045EE6AEDD2
:1041F0007CE5C8CF81E0C9CF9093D1018093D001F5
:10420000089590935404809353040895E0915304C7
:10421000F0915404309729F00190F081E02D099538
:10422000089580E00895E0915304F091540430978C
:1042300099F020912D01222359F020917C0427FF31
:1042400007C0DC012C9111962C93119726E02C933A
:104250000280F381E02D09950895E0915304F091D7
:104260005404309739F022E0DC012C930480F5816E
:10427000E02D09950895209151043091520428179A
:10428000390771F09093520480935104E0915304E4
:10429000F0915404309721F00680F781E02D0995C4
:1042A000089520914F04309150042817390771F078
:1042B0009093500480934F04E0915304F091540480
:1042C000309721F00084F185E02D09950895FC01D7
:1042D000329680912D01882321F080917C049EE10B
:1042E00087FF96E080E0915008F408952191222301
:1042F000D1F38F5FF8CF662301F120912D012223A6
:10430000F1F020917C0427FF1AC0462F4695469570
:1043100046954E3190F4677021E030E002C0220FE4
:10432000331F6A95E2F7840F911DFC01828190E0B2
:104330002823392381E0232B69F480E00895FC01D0
:10434000329608962191261721F0E817F907D1F740
:10435000F4CF81E008959C01FC0132969FEF80E04C
:104360004191461751F09F3F19F4411101C0982F18
:104370008F5F8630A9F79F3F09F40895290F311DFB
:1043800097FD3A95F90162830895FC0132960896EB
:104390002191261303C0DF0111971C92E817F9073A
:1043A000B9F70895E62FE695E695E695EE3168F4BF
:1043B000E80FF92FF11D677021E030E001C0220FF6
:1043C0006A95EAF78281822B82830895E62FE6952B
:1043D000E695E695EE3170F4E80FF92FF11D677060
:1043E00021E030E001C0220F6A95EAF72095828132
:1043F00028232283089520912D01222339F0209132
:104400007C0427FF03C00E94D22108950E94AB21A3
:10441000089520912D01222339F020917C0427FF5B
:1044200003C00E94E62108950E94C5210895FC0161
:10443000329680912D01882351F080917C0487FF72
:1044400006C08EE1DF011D928A95E9F7089586E0A6
:10445000F9CF46E050E00E946E2B21E0892B09F451
:1044600020E0822F089508950E943322089581113B
:1044700006C081E0809355040E943422089582E0B2
:10448000F9CF83E0809355040E94342208950E945E
:104490003722089581E0809355040E9434220895C4
:1044A0000E944A220895089508950E945422089572
:1044B000089508950E9453220895CF930E94582290
:1044C0000E94DA110E945922C0E08C2F0E94FE1037
:1044D000892B31F4CF5FC530C1F780E0CF910895CB
:1044E00081E0FCCF85B7806885BF85B7806885BFD0
:1044F00008951F921FB61F9211248F939F93AF931D
:10450000BF9380915604811113C0809188059091CA
:104510008905A0918A05B0918B054196A11DB11D19
:104520008093880590938905A0938A05B0938B05A5
:10453000BF91AF919F918F911F901FBE1F901895B3
:1045400080919005843031F10E94BA031092560494
:1045500088E190E020E40FB6F894A895809360007D
:104560000FBE2093600083B7817F846083BF83B7D1
:10457000816083BF7894889583B78E7F83BF0FB6A1
:10458000F894A895809160008861809360001092F3
:1045900060000FBE08950E9453070E94C40308954F
:1045A00082E084BD93E095BD9AEF97BD80936E0045
:1045B00008952FB7F8948091880590918905A0916E
:1045C0008A05B0918B052FBF08952FB7F89460919D
:1045D00088057091890580918A0590918B052FBF80
:1045E00008959C014FB7F8948091880590918905B2
:1045F000A0918A05B0918B054FBF821B930B089544
:1046000078941F921FB61F9211248F939F93AF939C
:10461000BF938091880590918905A0918A05B091FA
:104620008B050196A11DB11D809388059093890586
:10463000A0938A05B0938B05BF91AF919F918F9105
:104640001F901FBE1F90189581E08093E00080E2CC
:104650008093D8001092C9008FE19EE40197F1F792
:1046600000C0000087E090EBDC01809399059093F7
:104670009A05A0939B05B0939C0588E19CE00FB63A
:10468000F894A895809360000FBE90936000FFCFD0
:1046900088E19CE00FB6F894A895809360000FBE67
:1046A00090936000FFCF80917A04089508959C0153
:1046B00082E08093E9009FEF8091E800915085FDB2
:1046C00006C085ED8A95F1F700009111F5CF809134
:1046D000E80085FF0CC050E040E066E070E0C901F2
:1046E0000E949C258091E8008E778093E8000895D1
:1046F000CF93DF93EC0180912D018823B1F180915C
:104700007C0487FF32C060E282E08093E9008FEF93
:104710009091E800815095FD06C095ED9A95F1F7CE
:1047200000008111F5CF8091E80085FF1BC08091CA
:104730002D0170E050E040E0811104C050E040E005
:1047400068E070E0CE010E949C258091E8008E77A1
:104750008093E80080E2FE01AAE5B4E001900D92AA
:104760008A95E1F7DF91CF91089568E081E0CDCFA0
:104770008093570470935904609358048091900576
:10478000843001F582E08093E9008FEF9091E8009A
:10479000815095FD06C095ED9A95F1F700008111C5
:1047A000F5CF8091E80085FF0DC050E040E063E068
:1047B00070E087E594E00E949C258091E8008E7768
:1047C0008093E8000895BC0184E00E94B823089516
:1047D000BC0183E00E94B823089580918F05811168
:1047E00009C00E942C270E9489278091E2008460E2
:1047F0008093E200089510928F0508950E944A2246
:10480000089560918C0581E0611101C080E00E94F3
:10481000412208959091900581E0943009F080E064
:1048200060918C050E944722089542E061EC81E08E
:104830000E94A82642E261EC82E00E94A8269091A4
:10484000900581E0943009F080E060918C050E9431
:104850003722089580919205833009F461C030F4C5
:104860008130D1F1823009F49EC008958A3009F474
:104870008AC08B3009F46FC0893009F050C0809134
:104880009105813209F04BC0809195059091960574
:10489000029708F044C08091E800877F8093E80089
:1048A0008091E80082FF37C09091F3008091F20080
:1048B000029731F48091F100813011F0863021F4BB
:1048C0008091F10080937A048091E8008B77809347
:1048D000E8000E94DC2623C080919105813AF9F41A
:1048E0008091E800877F8093E80080919505909102
:1048F0009605892B61F460E28AE594E070E00E94FD
:10490000EB258091E8008B778093E800089560E0C4
:1049100090E080E0F3CF809190058111C1CF0895A0
:1049200080919105813AD9F78091950590919605EE
:10493000892BA9F78091E800877F8093E800809118
:10494000E80080FFFCCF80912D018093F1008091E1
:10495000E8008E77BCCF80919105813201F780917C
:10496000950590919605892BD1F68091E800877F77
:104970008093E8000E94DC268091930580932D01AE
:104980000E945307089580919105813241F68091EC
:10499000E800877F8093E8000E94DC2680919405E0
:1049A00080937B04089580919105813A09F0B7CFF7
:1049B0008091E800877F8093E8008091E80080FF85
:1049C000FCCF80917B04C1CF84B7877F84BF0FB6B3
:1049D000F894A8958091600088618093600010929F
:1049E00060000FBE80E890E00FB6F89480936100FD
:1049F000909361000FBE0E94502208950E942C27C0
:104A00000E948927E2EEF0E08081846080837894C0
:104A10000E94082A089581E291E00E9401210895F0
:104A200080919005853031F480919005853019F0A2
:104A30000E94CB2208950E94A02280918E05882397
:104A400099F30E945D22882379F30E9486250E94B3
:104A50005307EACF08950E942E250895292F332762
:104A60002330310519F168F42130310509F444C0CF
:104A70002230310509F445C090E080E030E020E0CC
:104A800025C02132310549F122323105A9F780E4F0
:104A900090E023E235E061157105C1F086EB90E00E
:104AA0002DE634E06130710589F0E6CF9927813039
:104AB000910581F0009729F00297F1F6E2EFF3E01B
:104AC00002C0ECE1F4E0849190E09F01FA013183AF
:104AD00020830895E0E1F4E0F6CF89E090E022E35E
:104AE00034E06115710591F389E090E02BE434E046
:104AF0006130710559F3C0CF82E190E02BE534E0DD
:104B0000E5CF8BE390E020E234E0E0CF80E189BDA7
:104B100082E189BD09B400FEFDCF8091D8008F7D70
:104B20008093D8008091E00082608093E0008091C3
:104B3000E00081FDFCCF0895AF92BF92CF92DF924B
:104B4000FF920F931F93CF93DF936C01EB018A01C8
:104B50000E94FB26F82E811123C00115110539F0A2
:104B6000F80180819181C81BD90BC80ED91EB12CC8
:104B7000A12C2097A9F08091E80085FD22C08091AA
:104B8000E8008E778093E80001151105A1F0F80187
:104B900080819181A80EB91EB182A08285E0F82E95
:104BA0008F2DDF91CF911F910F91FF90DF90CF90CC
:104BB000BF90AF9008950E94FB268823D1F2F82E73
:104BC000EFCFF60181916F018093F1002197FFEF04
:104BD000AF1ABF0ACECFFC0180919705909198053E
:104BE00086179707A0F06115710529F49091E800E8
:104BF0009E779093E80090E06115710551F4911152
:104C000008C08091E80082FF34C080E00895BC01B4
:104C1000F2CF809190058823C1F18530C1F1809158
:104C2000E80083FD30C08091E80082FDEACF8091EA
:104C3000E80080FFE1CF8091F3002091F200382F4F
:104C40006115710519F02830310558F091E02830D0
:104C5000310509F090E02091E8002E772093E800DC
:104C6000CBCF81918093F100615071092F5F3F4F4D
:104C7000E7CF80919005882341F0853041F0809105
:104C8000E80083FFBECF81E0089582E0089583E0CD
:104C90000895FC01809197059091980586179707D4
:104CA000A0F06115710529F48091E8008E7780935A
:104CB000E80090E06115710551F4911108C08091F0
:104CC000E80082FF35C080E00895BC01F2CF8091FA
:104CD00090058823C9F18530C9F18091E80083FDF2
:104CE00031C08091E80082FDEACF8091E80080FF2A
:104CF000E1CF8091F3002091F200382F611571050A
:104D000019F02830310558F091E02830310509F0CC
:104D100090E08091E8008E778093E800CBCF84917B
:104D20008093F1003196615071092F5F3F4FE6CFBC
:104D300080919005882341F0853041F08091E80012
:104D400083FFBDCF81E0089582E0089583E0089558
:104D5000982F973028F08F708093E90081E00895B4
:104D60009093E900242F762F50E0981731F070913E
:104D7000EC002091ED005091F00021FD02C09F5FFA
:104D8000E8CF3091EB003E7F3093EB003091ED00A7
:104D90003D7F3093ED003091EB0031603093EB00BC
:104DA0007093EC002093ED005093F0002091EE0002
:104DB00027FDE5CF80E008958091910587FF13C01E
:104DC0008091E80082FF06C08091E8008B77809395
:104DD000E80004C0809190058111F2CF0895809180
:104DE00090058823D9F38091E80080FFF8CF809167
:104DF000E8008E77ECCF2091E4003091E50095E655
:104E0000A9012091EC00822F817020FF06C08091C3
:104E1000E80080FF06C080E008952091E80022FDB0
:104E20001AC080919005882389F0853089F080919F
:104E3000EB0085FD0FC02091E4003091E5004217A2
:104E40005307F9F29150E1F684E0089582E0089565
:104E500083E0089581E008950E949B270E94A32784
:104E6000E0EEF0E0808181608083E8EDF0E0808119
:104E70008F77808319BCA7EDB0E08C918E7F8C93E7
:104E800080818F7E808310928F0508950F931F93EA
:104E9000CF93DF930E949B270E94A327C8EDD0E009
:104EA00088818F77888388818068888388818F7DD7
:104EB000888319BC1092900510928C0510928E0573
:104EC00010928D0500EE10E0F80180818B7F8083C9
:104ED00088818160888342E060E080E00E94A826AB
:104EE000E1EEF0E080818E7F8083E2EEF0E0808171
:104EF00081608083808188608083F80180818E7FDB
:104F00008083888180618883DF91CF911F910F9189
:104F10000895E8EDF0E080818F7E8083E7EDF0E09A
:104F200080818160808384E082BF81E080938F05EF
:104F30000E9446270895E8EDF0E080818E7F80830F
:104F40001092E20008951092DA001092E1000895A4
:104F50001F920F920FB60F9211242F933F934F93EE
:104F60005F936F937F938F939F93AF93BF93EF93D1
:104F7000FF938091E10082FF0BC08091E20082FFED
:104F800007C08091E1008B7F8093E1000E94072A97
:104F90008091DA0080FF19C08091D80080FF15C091
:104FA0008091DA008E7F8093DA008091D90080FFB3
:104FB00096C080E189BD82E189BD09B400FEFDCFC4
:104FC00081E0809390050E94ED238091E10080FFB5
:104FD00019C08091E20080FF15C08091E2008E7FB1
:104FE0008093E2008091E20080618093E2008091F2
:104FF000D80080628093D80019BC85E0809390052A
:105000000E9401248091E10084FF2BC08091E20086
:1050100084FF27C080E189BD82E189BD89B5982FD1
:10502000917080FFFBCF8091D8008F7D8093D80056
:105030008091E1008F7E8093E1008091E2008F7E7D
:105040008093E2008091E20081608093E200809191
:105050008C05882309F449C084E0809390050E9460
:105060000A248091E10083FF29C08091E20083FF40
:1050700025C08091E100877F8093E10082E08093EA
:10508000900510928C058091E1008E7F8093E10065
:105090008091E2008E7F8093E2008091E200806147
:1050A0008093E20042E060E080E00E94A8268091C8
:1050B000F00088608093F0000E94FE23FF91EF9142
:1050C000BF91AF919F918F917F916F915F914F9120
:1050D0003F912F910F900FBE0F901F90189519BC04
:1050E000109290050E94FB2370CF8091E30087FD12
:1050F00093E090939005B3CF1F920F920FB60F924B
:1051000011242F933F934F935F936F937F938F93CC
:105110009F93AF93BF93CF93DF93EF93FF93D09180
:10512000E900DF708091EC00C82FC17080FDC0E8FD
:105130001092E9008091F000877F8093F0007894CE
:105140000E94C0281092E9008091F000886080934E
:10515000F000CD2BCF70C093E900FF91EF91DF916C
:10516000CF91BF91AF919F918F917F916F915F91FF
:105170004F913F912F910F900FBE0F901F90189558
:10518000AAE2B0E0E6ECF8E20C94DD2A81E995E0D1
:105190002091F100FC012193CF01F5E089399F07AF
:1051A000B9F70E942A248091E80083FF1EC18091F4
:1051B0009105909192059A3008F017C1E92FF0E01F
:1051C000E051F44D0C94972A803899F0823809F018
:1051D0000CC1809195058F70873008F006C18093CF
:1051E000E9008091EB0085FB882780F91092E900A7
:1051F00006C080918D0590918E05911182609091ED
:10520000E800977F9093E8008093F1001092F100FE
:105210008091E8008E77E5C0882309F4D3C08230FE
:1052200009F0E3C0809193058111D6C08091950566
:105230008F702FEF280F263008F0D7C08093E90039
:105240002091EB0020FFC8C0933031F48091EB0037
:1052500080628093EB00C0C09091EB0090619093CE
:10526000EB0021E030E001C0220F8A95EAF720939D
:10527000EA001092EA008091EB008860EACF811189
:10528000B4C0109193051F778091E3008078812B43
:105290008093E3008091E800877F8093E8000E947C
:1052A000DC268091E80080FFFCCF8091E3008068DD
:1052B0008093E30082E0111183E08093900595C014
:1052C0008058823008F091C08091930590919405A8
:1052D0008C3D23E09207A1F583E08A838AE28983EB
:1052E0004FB7F894DE01139620E03EE051E2E32F41
:1052F000F0E050935700E49120FF03C0E295EF7077
:105300003F5FEF708E2F90E0EA30C0F0C7968D932C
:105310009D932F5F243159F74FBF8091E800877F1D
:105320008093E8006AE270E0CE0101960E94EB25CE
:105330008091E8008B778093E80057C0C096E7CF54
:105340006091950570919605AE014F5F5F4F0E9489
:105350002B25BC01892B09F448C09091E800977F68
:105360009093E80089819A810E944926E1CF803894
:10537000E1F58091E800877F8093E80080918C05BB
:105380008093F10045CF811130C090919305923008
:1053900060F58091E800877F8093E80090938C050A
:1053A0000E94DC2680918C05882311F084E005C0E2
:1053B0008091E30087FDFACF81E0809390050E9401
:1053C000152413C080919305813079F481E09330E6
:1053D00009F080E080938E051092E9008091E8004A
:1053E000877F8093E8000E94DC268091E80083FF9D
:1053F0000AC08091E800877F8093E8008091EB00ED
:1054000080628093EB00AA96E3E00C94F92A089559
:10541000CF93809190058823A1F0C091E900CF70CF
:105420009091EC00892F817090FD80E8C82B10923C
:10543000E9008091E80083FD0E94C028CF70C093EE
:10544000E900CF910895DB018F939F930E94BB2ABF
:10545000BF91AF91A29F800D911DA39F900DB29F10
:10546000900D11240895991B79E004C0991F961797
:1054700008F0961B881F7A95C9F78095089587FBD9
:10548000082E062687FD819567FD61950E94332AC7
:105490000EF4919507FC81950895AA1BBB1B51E161
:1054A00007C0AA1FBB1FA617B70710F0A61BB70B94
:1054B000881F991F5A95A9F780959095BC01CD0139
:1054C000089597FB072E16F4009407D077FD09D0B6
:1054D0000E944D2A07FC05D03EF4909581959F4F80
:1054E0000895709561957F4F0895A1E21A2EAA1B29
:1054F000BB1BFD010DC0AA1FBB1FEE1FFF1FA21784
:10550000B307E407F50720F0A21BB30BE40BF50B80
:10551000661F771F881F991F1A9469F76095709509
:10552000809590959B01AC01BD01CF010895EE0FD0
:10553000FF1F0590F491E02D09940E94A52A3323C2
:1055400012F48A1B9B0B0C94B62AA29FB001B39F46
:10555000C001A39F700D811D1124911DB29F700D7C
:10556000811D1124911D08950E94A52AB7FF089559
:10557000821B930B08950E94A52AA59F900DB49FAE
:10558000900DA49F800D911D11240895B7FF0C94D8
:10559000BB2A0E94BB2A821B930B08952F923F9235
:1055A0004F925F926F927F928F929F92AF92BF9233
:1055B000CF92DF92EF92FF920F931F93CF93DF93DF
:1055C000CDB7DEB7CA1BDB0B0FB6F894DEBF0FBE3C
:1055D000CDBF09942A88398848885F846E847D8489
:1055E0008C849B84AA84B984C884DF80EE80FD808B
:1055F0000C811B81AA81B981CE0FD11D0FB6F89401
:10560000DEBF0FBECDBFED0108958F929F92AF9286
:10561000BF92CF92DF92EF92FF92CF93DF93EC0194
:10562000688179818A819B81611571058105910568
:1056300021F464E279ED8BE597E02DE133EF41E071
:1056400050E00E94C32B49015A019B01AC01A7EA1B
:10565000B1E40E94BB2A6B017C01ACEEB4EFA50162
:1056600094010E94C92ADC01CB018C0D9D1DAE1D49
:10567000BF1DB7FF03C00197A109B0488883998374
:10568000AA83BB839F77DF91CF91FF90EF90DF904C
:10569000CF90BF90AF909F908F9008950E94052B60
:1056A000089580E091E00E94052B0895B0E0A0E00D
:1056B0008093000190930101A0930201B093030134
:1056C0000895FC014150504030F001900616D1F78A
:1056D0003197CF010895882799270895FB01DC01B0
:1056E00004C08D910190801921F441505040C8F7B9
:1056F000881B990B0895F999FECF92BD81BDF89A48
:10570000992780B50895A6E1B0E044E050E00C94FC
:10571000B52BA8E1B0E042E050E00C94B52B262F69
:10572000F999FECF92BD81BDF89A019700B4021697
:1057300039F01FBA20BD0FB6F894FA9AF99A0FBE45
:1057400008950396272F0E94902B0E948F2B252FC0
:105750000E94902B242F0C94902B0196272F0E94AF
:10576000902B0C948F2BDC01CB01FC01F999FECF1F
:1057700006C0F2BDE1BDF89A319600B40D924150D9
:105780005040B8F70895052E97FB1EF400940E9430
:10579000DA2B57FD07D00E94752A07FC03D04EF480
:1057A0000C94DA2B50954095309521953F4F4F4FF3
:1057B0005F4F089590958095709561957F4F8F4FBD
:1057C0009F4F0895F894FFCF2305230554055405F2
:1057D000E105FD058305830508069406A306A306D7
:1057E000E4280C29F5290C29F5293F296029F529F8
:0457F000B729C329E9
:1057F400010000006802280850011E0A140101017A
:1058040002005000505001191A1B1C1D1E1F20219C
:1058140022532378235723E823E323562301E2006A
:10582400E900EA00B500B600B700CD008301CC0062
:105834008A019201940121022302240225022602F4
:1058440027022A02B300B4006F007000818283E251
:1058540000E900EA00B500B600B700CD008301CC32
:10586400008A0192019401210223022402250226C6
:105874000227022A02B300B4006F00700081828301
:10588400909192939594969734F7F6F5F4F1F0305D
:105894003132333700010202020206060609090901
:1058A4000909090F0F0F0F0F0F15151518191919DD
:1058B4001919191919191923242525252525250010
:00000001FF
